:020000040000FA
:04000000E9EF0DF027
:08000800056ED8CF06F0E0CF31
:1000100007F00001E9CF0DF0EACF08F0E1CF09F0D9
:10002000E2CF0AF0D9CF0BF0DACF0CF0F3CF14F017
:10003000F4CF15F0FACF16F000C00FF001C010F0A9
:1000400002C011F003C012F004C013F0A0AA2CEFFC
:1000500000F0A1BA87EF07F00FC000F010C001F068
:1000600011C002F012C003F013C004F00DC0E9FF8C
:1000700008C0EAFF088E09C0E1FF0AC0E2FF0BC01A
:10008000D9FF0CC0DAFF14C0F3FF15C0F4FF16C08F
:10009000FAFF055007C0E0FF06C0D8FF1000F76A5E
:1000A000AE0FF66E000EF7220900F55012000003A5
:1000B000FFFFFFFFFFFFFFFFFFFFFFFFFFFF08AE98
:1000C00003D0F2CF0EF0F29EF76AE00FF66E000E4C
:1000D000F7220900F55008AE02D00EBEF28E1200D3
:1000E00040000800000000000000000000000000C8
:1000F0000000000000000000000000000000000000
:10010000F76A100FF66E010EF7220900F550120083
:100110000600FF0901A101190129081580257F7535
:10012000089508810819012908750895089108C0E3
:10013000F76A400FF66E010EF7220900F550120023
:100140000000F76A520FF66E010EF7220900F55013
:1001500012002000F76A640FF66E010EF722090004
:10016000F550120009022900010100C03209040003
:100170000002030000000921000100012220000705
:100180000581030800010705010308000100F76A63
:100190009E0FF66E010EF7220900F55012000100C5
:1001A000F76AB00FF66E010EF7220900F550120043
:1001B0001200F76AC20FF66E010EF7220900F55021
:1001C00012001201100100000040610447100001FC
:1001D00001020001F76AE40FF66E010EF722090032
:1001E000F5501200040309040803540044004500BC
:1001F0002C03540065006300680044006500730030
:10020000690067006E0020004D006F0064007500FB
:100210006C0065002000300034003700F2CF0EF093
:10022000F29EF76A360FF66E020EF7220900F550BD
:100230000EBEF28E12000A0A0D20303437202D2017
:10024000546F756368506164204D6F64756C6520F0
:100250000A0A0D00F2CF0EF0F29EF76A6E0FF66EEC
:10026000020EF7220900F5500EBEF28E1200202A6F
:100270002A206C6F775F54483D254C780000F2CF00
:100280000EF0F29EF76A980FF66E020EF722090042
:10029000F5500EBEF28E12002070726F78696D6993
:1002A00074793D254C780000F2CF0EF0F29EF76A8B
:1002B000C20FF66E020EF7220900F5500EBEF28E46
:1002C00012000D0A2D2D3E20526563656976656426
:1002D00020646174613A20307825582030782558A0
:1002E0000A0D0000F2CF0EF0F29EF76AFE0FF66ED6
:1002F000020EF7220900F5500EBEF28E12000D0A12
:100300000A55534220636F6E6E65637465642C20DA
:1003100077616974696E6720666F7220656E756DAE
:1003200065726174696F6E2E2E2E0000F2CF0EF092
:10033000F29EF76A460FF66E030EF7220900F5509B
:100340000EBEF28E12000D0A0A55534220646973E4
:10035000636F6E6E65637465642C20776169746980
:100360006E6720666F7220636F6E6E656374696F6F
:100370006E2E2E2E0000F2CF0EF0F29EF76A900F36
:10038000F66E030EF7220900F5500EBEF28E120033
:100390000D0A0A55534220656E756D65726174656C
:1003A000642062792050432F484F53540000F2CF0D
:1003B0000EF0F29EF76AC80FF66E030EF7220900E0
:1003C000F5500EBEF28E12000D0A0A5553422075EA
:1003D0006E656E756D65726174656420627920501A
:1003E000432F484F53542C2077616974696E6720FE
:1003F000666F7220656E756D65726174696F6E2EC1
:100400002E2E00006D92699468A402D06894FCD7E7
:1004100092EF07F0400E0401016F040E036F100EFF
:10042000026F880E006F046B040E076F500E066F8C
:100430000001000C70A002D0EDDF7090689A9BEF75
:1004400007F06A6A6892A1EF07F0036A8551700F9E
:10045000E96E0F0E0320EA6EEF6A8551080DF35026
:10046000876BE96E040E8725EA6EEF6A8551080DE9
:10047000F350876B866F040E8627000E872386C095
:10048000E9FF040E8725EA6EEF6A000C010E846F07
:1004900084510F0805E384C085F0D7DF842BF8D79B
:1004A000000C7A6B7A530AE1036A7A512B0FE96EDA
:1004B000000E0320EA6EEF6A7A2BF4D7206A010E51
:1004C000216E1F6A000C689600D000D000D0000C8E
:1004D0006A6A686A9F0E6B6E3D0E696E6E6AD6DF41
:1004E000E0DF160E706E68A602D0EDDFFCD76D98C7
:1004F00091DF030E266EA7EF07F0698468986D827E
:10050000ADEF07F0689CB3EF07F07FC027F0000C59
:10051000FF0E276E000C7D6B2A5242E07D513F0892
:100520003FE32250FC0F2BE2040FDAEF02F0036AE4
:100530002950F2CF7FF0F29E0DDE7FBFF28E7E6FEC
:100540001ED0036A2950F2CF7FF0F29ED9DD7FBF23
:10055000F28E7E6F14D0036A2950F2CF7FF0F29EA4
:1005600039DE7FBFF28E7E6F0AD0036A2950F2CF48
:100570007FF0F29E1EDE7FBFF28E7E6F00D0292AB2
:100580002A067D517D2B036A500F016E000E032257
:1005900001C0E9FF040E0324EA6E7EC0EFFFBCD762
:1005A0002A5204E17D51400801E01F6A7DC07FF0BE
:1005B000ACDF000CE824F76AF736CF0FF66E050EB5
:1005C000F7220A00F550FA6E0800F550F96E2E0574
:1005D000420556056A05296A226A04011351010A77
:1005E000000109E0030A0CE0010A0DE0220A22E002
:1005F000030A3FE065D0120E2A6E030E226E62D00F
:10060000290E2A6E5FD0020E226E036A0401125177
:10061000230FE96E000E0320EA6EEFCF29F0036A84
:100620002950F2CF7DF0F29E0001D4DD7DBFF28E25
:100630002A6E48D0D89004011235036AF2CF7DF0BB
:10064000F29E0001ADDD0900F5CF03F07DBFF28E13
:10065000296E293C01D00BD0036A2950F2CF7DF0DE
:10066000F29E78DD7DBFF28E2A6E2CD002D050DF54
:1006700035D0D89004011435036AF2CF7DF0F29E94
:10068000000156DD0900F5CF03F07DBFF28E296E23
:10069000293C01D013D0010E226ED89004011435EC
:1006A000036AF2CF7DF0F29E00014BDD0900F5CF29
:1006B00003F07DBFF28E2A6E05D002D029DF0ED066
:1006C00027DF0CD00401175305E12A50165D02E222
:1006D00016C42AF0010E1F6E00011DDF000C7C53B2
:1006E00004E1040E266ED2DECFD0050E266E040E77
:1006F0007F6F900E7E6F010E7D6F7D510F08D8A029
:10070000C3D07DC085F0A1DE806B036A7D51F2CF3E
:1007100084F0F29EC4DC84BFF28EFF0857E0040E22
:10072000806FD8907D35036AF2CF84F0F29EC7DCEB
:100730000900F5CF03F084BFF28E816F03C082F011
:100740007D51080DF350856B846F010E8425016E79
:10075000000E8521036E01C0E9FF040E0324EA6E3A
:1007600081C0EFFF7D51080DF350856B846F020E41
:100770008425016E000E8521036E01C0E9FF040E81
:100780000324EA6E7FC0ECFFED527EC0EFFFD890ED
:100790007D35036AF2CF84F0F29E91DC0900F5CF3B
:1007A00003F084BFF28E7E2703507F23880E836F71
:1007B00082B1838182B383837D51080DF350856BB1
:1007C000E96E040E8525EA6E83C0EFFF036A7D5152
:1007D000F2CF84F0F29E63DC84BFF28EFF0839E032
:1007E00080837D51080DF350856B846F040E842740
:1007F000000E8523020E8425016E000E8521036EF6
:1008000001C0E9FF040E0324EA6E7FC0ECFFED5245
:100810007EC0EFFFD8907D35036AF2CF84F0F29E60
:100820004EDC0900F5CF03F084BFF28E7E27035023
:100830007F237D51080DF350856B846F040E842750
:10084000000E852384C0E9FF040E8525EA6E400E64
:10085000EF6E8051060802E10E0E806F036A7D5133
:10086000F2CF84F0F29E1BDC84BFF28E0108D8A484
:100870008089036A7D51700FE96E0F0E0320EA6EC6
:1008800080C0EFFF7D2B39D790EF04F004011151A8
:1008900000010DE0010A14E0020A1EE0060A27E04A
:1008A000030A2CE00E0A2CE0010A30E03DD021C002
:1008B00050F40401516B020E00017F6F26DE36D02A
:1008C0000401122D06D0010E211600017F6B1DDEE2
:1008D00002D000011DDE2AD00401122D05D0218294
:1008E00000017F6B12DE02D0000112DE1FD0020E6B
:1008F0001F6E12C428F07F6B08DE18D06CDE16D095
:1009000020C050F4010E7F6F00DE10D004011251A0
:10091000010808E312C420F012C47CF00001DFD605
:100920007F6BF3DD000102D0F3DD00D0CBEF05F0EB
:1009300020C07CF004011151000107E00A0A0DE01B
:10094000010A2DE00D0A3DE03ED00401506B516BD1
:10095000020E00017F6FD9DD38D07C531EE0010EFE
:100960007C5D036AF2CF7DF0F29E11DC7DBFF28EDA
:10097000016E0401145DD8A002D000010ED0036AFC
:1009800014512B0FE96E000E0320EA6EEFCF50F4E6
:10099000010E00017F6FB9DD01D0BADD16D07C53A6
:1009A0000EE0036A040114512B0FE96E000E0320C0
:1009B000EA6E12C4EFFF00017F6BA7DD01D0A8DD56
:1009C00004D009DE02D0A4DD00D0CBEF05F07D918C
:1009D0007CBF7D817C9F7DA111D0036A7C51F2CFC9
:1009E0007EF0F29E4FEC00F07EBFF28EFF0802E137
:1009F000000E01D0010E016E11D010D0036A7C519F
:100A0000F2CF7EF0F29E4FEC00F07EBFF28EFF0838
:100A100002E1000E01D0010E016E00D083EF05F05F
:100A20007D917CBF7D817C9F7DA111D07C51080D83
:100A3000F3507F6B7E6F040E7E27000E7F237EC0F7
:100A4000E9FF040E7F25EA6E880EEF6E09D07C5117
:100A5000080DF3507F6BE96E040E7F25EA6EEF6A96
:100A600092EF05F07D917CBF7D817C9F7DA111D0AF
:100A70007C51080DF3507F6B7E6F040E7E27000EB5
:100A80007F237EC0E9FF040E7F25EA6E840EEF6EA1
:100A90000AD07C51080DF3507F6BE96E040E7F2560
:100AA000EA6E840EEF6E98EF05F07D917CBF7D813C
:100AB0007C9F7DA111D07C51080DF350806B7F6F1E
:100AC000040E7F27000E80237FC0E9FF040E8025DF
:100AD000EA6EEFCF7EF00AD07C51080DF350806BA8
:100AE000E96E040E8025EA6EEFCF7EF07EAF02D075
:100AF0007EB502D0000E01D0010E016EA2EF05F00E
:100B000014C47CF064D7015229E004011151010A98
:100B1000000105E0020A09E0030A0DE01DD014C43B
:100B20007CF07ED77F6BF1DC19D014C47CF09AD7AF
:100B30007F6BEBDC13D00401506B516B14C47CF061
:100B40000001B3D7015204E0010E0401506F00010F
:100B5000020E7F6FDADC02D0DBDC00D0CBEF05F0D9
:100B60000401115100D00001D3DC00D0CBEF05F01F
:100B70001F6A040110517F0B000107E0010A06E023
:100B8000030A05E0230A04E004D080D6D1D6B8D702
:100B9000E7D7BEDC00D0F5EF06F07C51080DF3502E
:100BA000826BE96E040E8225EA6EEFCF7EF07D51F6
:100BB000020806E17EAD02D07D6B02D0010E7D6F92
:100BC0007D51030813E1840E7E6F7C51080DF350B4
:100BD000826B816F040E8127000E822381C0E9FFA2
:100BE000040E8225EA6E840EEF6E07D07D2D03D0B1
:100BF000C80E7E6F02D0880E7E6FD8907C35036A57
:100C0000F2CF81F0F29E5FEC00F00900F5CF03F027
:100C100081BFF28E7F6F03C080F07C51080DF350CE
:100C2000826B816F010E8125016E000E8221036EA1
:100C300001C0E9FF040E0324EA6E7FC0EFFF80B11C
:100C40007E8180B37E837C51080DF350826BE96E08
:100C5000040E8225EA6E7EC0EFFF000C036A81510C
:100C6000700FE96E0F0E0320EA6EEF5212E0815111
:100C7000080DF350836B826F040E8227000E8323CE
:100C800082C0E9FF040E8325EA6EEFCF82F082AFC7
:100C900002D0000E01D0010E016E000C7CC081F06C
:100CA000DDDF015262E07C51080DF350826B816FF1
:100CB000040E8127000E8223010E8125016E000E95
:100CC0008221036E01C0E9FF040E0324EA6E7DC099
:100CD000EFFF7F51020817E17C51080DF350826B42
:100CE000816F040E8127000E822381C0E9FF040E6C
:100CF0008225EA6EEFCF80F080AD02D07F6B02D00C
:100D0000010E7F6F13D07F51040810E17C51080D54
:100D1000F350826BE96E040E8225EA6EEFCF80F00D
:100D200080AD03D0010E7F6F01D07F6B7F2D03D08C
:100D3000C80E806F02D0880E806F7EB180817EB336
:100D400080837C51080DF350826B816F040E8127E4
:100D5000000E822381C0E9FF040E8225EA6E80C066
:100D6000EFFF010E016E03D000D0000E016E000CEB
:100D70007C5302E10AEC02F0000C7DC06EFF7D5353
:100D800003E0040E266E02D0020E266ECDEF06F0B2
:100D9000206A1F6A28C07DF0F0D7DAEF06F07C5396
:100DA00009E11F2C03D08BEC02F004D01F50020885
:100DB00001E1EED7000C6C307A6F7A337A331F0E74
:100DC0007A176C5240E1040100513C0B00017B6F2B
:100DD000430E04010017000163EC02F07B5134085C
:100DE0001BE10401046B0001C3D66D98273C05D0BC
:100DF0007C6B030E7D6FD1DE0ED07C6B020E7D6F9F
:100E0000CCDE2750FE0807E07C6B7E6B27C07DF0B0
:100E1000040E7F6F43DF16D07B51040813E17C6B17
:100E2000A7DF7C6B020E7D6FB8DE2750FE080AE05C
:100E3000273C01D007D07C6B7E6B27C07DF0010E74
:100E40007F6F2CDF62D06C50040818E1430E040160
:100E50000417000163EC02F0FF0E276E7C6B9FDF2E
:100E6000273C01D008D07C6B7E6B27C07DF0020E42
:100E70007F6F14DF02D00AEC02F047D06CB41DD0B3
:100E80007A51080DF3507D6B016E040E7D25036EC3
:100E90007A51080DF3507F6BE96E040E7F25EA6EE0
:100EA000EF50430B03C0EAFF01C0E9FFEF6E63ECB4
:100EB00002F07AC07CF05CDF28D07A51080DF35044
:100EC0007D6B7C6F040E7C27000E7D237CC001F0BF
:100ED000040E7D25036E7A51080DF3507F6B7E6FF3
:100EE000040E7E27000E7F237EC0E9FF040E7F25BF
:100EF000EA6EEF50430B03C0EAFF7CC0E9FFEF6EE0
:100F000063EC02F07AC07CF04ADFB9EF07F02652BA
:100F100001E135D0685233E068A404D069A402D05E
:100F200002EF02F06DA201D02AD068AA04D069AA0B
:100F300002D01AEF02F068A204D069A202D021EF19
:100F400002F068A004D069A002D068EF02F068A89F
:100F500004D069A802D07DEF02F068AC04D069AC7F
:100F600002D082EF02F0796B68A604D069A602D0A5
:100F700022D701D004D07951792B0308F5E2A19A48
:100F80002CEF00F06D6A696A080E6F6E945030099C
:100F9000946E266A186AF2BE188EF29E51EC02F028
:100FA00018BEF28ED5EF07F0EDD7FAEF07F0186A0A
:100FB000F2BE188EF29E51EC02F018BEF28E6D6AEF
:100FC000140E6F6E696A6D86010E266EEBEF07F0E8
:100FD0006DB601D0ECD7262C0BD06DBA09D0686A5B
:100FE000696AA08AC00EF212110E696E020E266E98
:100FF000000CDAD7EDDF26500208FCE128EF0EF0F6
:101000009EA8FED7AD6E000C6E6B6F6B706B716B34
:10101000818600D000D00000819800D000D0000070
:10102000685306E169C06EF06A51E0096F6F07D03E
:10103000682D05D069C06EF06A51E4096F6F0F0E1C
:101040006D6F6D3D01D01BD0819600D000D00000A7
:101050006FC003F06EC002F06D51006E05E0D890D5
:1010600003320232002EFBD7025002A0819C02B054
:10107000818C818600D000D000006D07E2D76853D4
:1010800000E10F0E6D6F6D3D01D031D0819600D023
:1010900000D00000682D12D081AE0FD0036A010E7F
:1010A000026E6D51006E05E0D89002360336002EB8
:1010B000FBD7025070130350711313D0685311E122
:1010C0006CC003F06BC002F06D51006E05E0D8906B
:1010D00003320232002EFBD7025002A0819C02B0E4
:1010E000818C818600D000D000006D07CCD781882C
:1010F00070C001F071C002F0000CF2CF68F0F29EF7
:10110000010EA96EA69CA69EA680A85068BFF28E6E
:10111000616F612D04D0120E606F5F6E42D061511D
:10112000020804E1130E606F5F6E3BD0615103084B
:1011300004E1140E606F5F6E34D06151040804E165
:10114000150E606F5F6E2DD06151050804E1170E1A
:10115000606F5F6E26D06151060804E1190E606F62
:101160005F6E1FD06151070804E11A0E606F5F6E59
:1011700018D06151080804E11C0E606F5F6E11D039
:101180006151090804E11E0E606F5F6E0AD0615163
:101190000A0804E11F0E606F5F6E03D0170E606FC8
:1011A0005F6E686B6A6B696B040E6C6F6B6B2CDF28
:1011B000C70E006E002EFED700D0686B6A6B800EE3
:1011C000696F3F0E6C6FFF0E6B6F1EDF686B6A6B93
:1011D000810E696F2F0E6C6FFF0E6B6F15DF686BE2
:1011E0006A6B820E696F010E6C6F6B6B0DDF686B43
:1011F0006A6B830E696F60C06CF05FC06BF004DFD8
:10120000686B6A6B840E696F6C6B680E6B6FFCDECB
:10121000686B6A6B850E696F6C6B680E6B6FF4DEC2
:10122000686B6A6B860E696F6C6B800E6B6FECDEA1
:10123000686B6A6B870E696F6C6B800E6B6FE4DE98
:10124000686B6A6B880E696F3F0E6C6FBF0E6B6FB9
:10125000DBDE686B6A6B890E696F3F0E6C6FFF0E89
:101260006B6FD2DE686B6A6B8A0E696F030E6C6FF0
:101270006B6BCADE686B6A6B8B0E696F60C06CF05B
:101280005FC06BF0C1DE686B6A6B8C0E696F6C6B54
:10129000680E6B6FB9DE686B6A6B8D0E696F6C6B75
:1012A000680E6B6FB1DE686B6A6B8E0E696F6C6B6C
:1012B000800E6B6FA9DE686B6A6B8F0E696F6C6B4B
:1012C000800E6B6FA1DE686B6A6B900E696F3E0ECD
:1012D0006C6FFF0E6B6F98DE686B6A6B910E696FB7
:1012E0003F0E6C6FFF0E6B6F8FDE686B6A6B920E3A
:1012F000696F030E6C6F6B6B87DE686B6A6B930EA6
:10130000696F60C06CF05FC06BF07EDE686B6A6B0B
:10131000940E696F6C6B680E6B6F76DE686B6A6B30
:10132000950E696F6C6B680E6B6F6EDE686B6A6B27
:10133000960E696F6C6B800E6B6F66DE686B6A6B06
:10134000970E696F6C6B800E6B6F5EDE686B6A6BFD
:10135000980E696F3B0E6C6FFF0E6B6F55DE686BFE
:101360006A6B990E696F3F0E6C6FFF0E6B6F4CDEF0
:10137000686B6A6B9A0E696F030E6C6F6B6B44DE61
:10138000686B6A6B9B0E696F60C06CF05FC06BF03E
:101390003BDE686B6A6B9C0E696F6C6B680E6B6FE3
:1013A00033DE686B6A6B9D0E696F6C6B680E6B6FDA
:1013B0002BDE686B6A6B9E0E696F6C6B800E6B6FB9
:1013C00023DE686B6A6B9F0E696F6C6B800E6B6FB0
:1013D0001BDE686B6A6BA00E696F2F0E6C6FFF0EC1
:1013E0006B6F12DE686B6A6BA10E696F3F0E6C6FDC
:1013F000FF0E6B6F09DE686B6A6BA20E696F030EDE
:101400006C6F6B6B01DE686B6A6BA30E696F60C0FB
:101410006CF05FC06BF0F8DD686B6A6BA40E696FEF
:101420006C6B680E6B6FF0DD686B6A6BA50E696F95
:101430006C6B680E6B6FE8DD686B6A6BA60E696F8C
:101440006C6B800E6B6FE0DD686B6A6BA70E696F6B
:101450006C6B800E6B6FD8DD686B6A6BA80E696F62
:101460003F0E6C6FFF0E6B6FCFDD686B6A6BA90E62
:10147000696F3F0E6C6FFE0E6B6FC6DD686B6A6B3B
:10148000AA0E696F030E6C6F6B6BBEDD686B6A6BC7
:10149000AB0E696F60C06CF05FC06BF0B5DD686B60
:1014A0006A6BAC0E696F6C6B680E6B6FADDD686B51
:1014B0006A6BAD0E696F6C6B680E6B6FA5DD686B48
:1014C0006A6BAE0E696F6C6B800E6B6F9DDD686B27
:1014D0006A6BAF0E696F6C6B800E6B6F95DD686B1E
:1014E0006A6BB00E696F3F0E6C6FFF0E6B6F8CDD19
:1014F000686B6A6BB10E696F3F0E6C6FFB0E6B6FA2
:1015000083DD686B6A6BB20E696F030E6C6F6B6B79
:101510007BDD686B6A6BB30E696F60C06CF05FC097
:101520006BF072DD686B6A6BB40E696F6C6B680E82
:101530006B6F6ADD686B6A6BB50E696F6C6B680EFA
:101540006B6F62DD686B6A6BB60E696F6C6B800ED9
:101550006B6F5ADD686B6A6BB70E696F6C6B800ED0
:101560006B6F52DD686B6A6BB80E696F3F0E6C6F04
:10157000FF0E6B6F49DD686B6A6BB90E696F3F0ECA
:101580006C6FEF0E6B6F40DD686B6A6BBA0E696F44
:10159000030E6C6F6B6B38DD686B6A6BBB0E696F2B
:1015A00060C06CF05FC06BF02FDD686B6A6BBC0EC7
:1015B000696F6C6B680E6B6F27DD686B6A6BBD0EB5
:1015C000696F6C6B680E6B6F1FDD686B6A6BBE0EAC
:1015D000696F6C6B800E6B6F17DD686B6A6BBF0E8B
:1015E000696F6C6B800E6B6F0FDD686B6A6BC00E82
:1015F000696F3F0E6C6FFF0E6B6F06DD686B6A6B79
:10160000C10E696F3F0E6C6FBF0E6B6FFDDC686BB8
:101610006A6BC20E696F030E6C6F6B6BF5DC686BE7
:101620006A6BC30E696F60C06CF05FC06BF0ECDC7E
:10163000686B6A6BC40E696F6C6B680E6B6FE4DC71
:10164000686B6A6BC50E696F6C6B680E6B6FDCDC68
:10165000686B6A6BC60E696F6C6B800E6B6FD4DC47
:10166000686B6A6BC70E696F6C6B800E6B6FCCDC3E
:10167000686B6A6BC80E696F3F0E6C6FFF0E6B6F05
:10168000C3DC686B6A6BC90E696F3E0E6C6FFF0E30
:101690006B6FBADC686B6A6BCA0E696F030E6C6F96
:1016A0006B6BB2DC686B6A6BCB0E696F60C06CF001
:1016B0005FC06BF0A9DC686B6A6BCC0E696F6C6BFA
:1016C000680E6B6FA1DC686B6A6BCD0E696F6C6B1B
:1016D000680E6B6F99DC686B6A6BCE0E696F6C6B12
:1016E000800E6B6F91DC686B6A6BCF0E696F6C6BF1
:1016F000800E6B6F89DC686B6A6BD00E696F3F0E72
:101700006C6FFF0E6B6F80DC686B6A6BD10E696F5C
:101710003B0E6C6FFF0E6B6F77DC686B6A6BD20EE3
:10172000696F020E6C6F6B6B6FDC686B6A6BD30E4C
:10173000696F60C06CF05FC06BF066DC686B6A6BF1
:10174000D40E696F6C6B680E6B6F5EDC686B6A6BD6
:10175000D50E696F6C6B680E6B6F56DC686B6A6BCD
:10176000D60E696F6C6B800E6B6F4EDC686B6A6BAC
:10177000D70E696F6C6B800E6B6F46DC686B6A6BA3
:10178000D80E696F3F0E6C6FEF0E6B6F3DDC686BB0
:101790006A6BD90E696F3F0E6C6FFF0E6B6F34DC96
:1017A000686B6A6BDA0E696F050E6C6F6B6B2CDC05
:1017B000686B6A6BDB0E696F60C06CF05FC06BF0CA
:1017C00023DC686B6A6BDC0E696F6C6B680E6B6F89
:1017D0001BDC686B6A6BDD0E696F6C6B680E6B6F80
:1017E00013DC686B6A6BDE0E696F6C6B800E6B6F5F
:1017F0000BDC686B6A6BDF0E696F6C6B800E6B6F56
:1018000003DC686B6A6B696B200E6C6FB00E6B6FDC
:1018100004EC08F0686B6A6B010E696F6C6B6B6BA4
:1018200004EC08F0686B6A6B020E696F320E6C6F25
:10183000300E6B6F04EC08F0686B6A6B030E696F17
:10184000080E6C6FC80E6B6F04EC08F0686B6A6B67
:10185000040E696F080E6C6F320E6B6F04EC08F0AB
:10186000686B6A6B050E696F6C6B6B6B04EC08F050
:10187000686B6A6B060E696F6C6B6B6B04EC08F03F
:10188000686B6A6B070E696F6C6B010E6B6F04EC13
:1018900008F0686B6A6B010E696F0F0E6C6FFF0EBC
:1018A0006B6F04EC08F0000C6951070B006E693196
:1018B000016E013201321F0E011601506B25E96ED7
:1018C000000E6C21EA6E016A012A002A01D001365D
:1018D000002EFDD76A5303E00150EF1203D0011E22
:1018E0000150EF164CEF0EF06951070B006E693195
:1018F000016E013201321F0E011601506A25E96E98
:10190000000E6B21EA6EEFCF01F0002A01D0013208
:10191000002EFDD753EF0EF069BF10D00F0E006EF2
:10192000683900160A0E005C03E2300E002602D071
:101930006951002600509EA8FED7AD6E0F0E6817A5
:101940000A0E685D02E2300E02D0699F6951682775
:1019500068519EA8FED7AD6E000C2050016E000CA1
:10196000010E686FFADF01C069F068530CE066533E
:101970000AE16A6B6A5172EC01F06A2B00EC08F024
:101980002C0E6A5DF7E168530CE166530AE06A6B5E
:101990006A5196EC01F06A2B00EC08F02E0E6A5D9D
:1019A000F7E169530CE067530AE16A6B6A51BBECDB
:1019B00001F06A2B00EC08F01C0E6A5DF7E1695338
:1019C0000CE167530AE06A6B6A51D7EC01F06A2BAD
:1019D00000EC08F03A0E6A5DF7E168C066F069C095
:1019E00067F0D2EF0EF0036A6851700FE96E0F0EC8
:1019F0000320EA6EEF520DE06851080DF3506A6B58
:101A0000696FE96E040E6A25EA6EEFCF69F069AF7F
:101A100002D0000E01D0010E016ED9EF0EF06D5113
:101A2000080DF350786B776F020E7725016E000E6C
:101A30007821036E01C0E9FF040E0324EA6EECCFA7
:101A400003F0ED52EFCF72F003C073F06D51080D4B
:101A5000F350786B776F010E7725016E000E7821B9
:101A6000036E01C0E9FF040E0324EA6EEF50036A1F
:101A7000756F03C076F06D51080DF350786BE96E09
:101A8000040E7825EA6EEFCF74F074B1768174B3EA
:101A900076837651715D08E303E17051755D04E270
:101AA00076C071F075C070F06FC0EAFF6EC0E9FFDC
:101AB00073C0E2FF72C0E1FF71C002F070C001F0BC
:101AC000015202E0022A02D0025206E0E6CFEEFF07
:101AD000012EFCD7022EFAD770C001F071C002F0BF
:101AE0007DEF0DF068C06DF06AC06FF069C06EF0F8
:101AF0006CC071F06BC070F092D702C06CF001C086
:101B00006BF0186AF2BE188EF29E68C07CF0020E6E
:101B10007D6FCDEC05F018BEF28E6BC001F06CC08D
:101B200002F0E4EF0EF0186AF2BE188EF29E68C062
:101B300081F02EEC06F018BEF28E015246E068519C
:101B4000080DF350716B706F040E7027000E712337
:101B5000020E7025016E000E7121036E01C0E9FFB7
:101B6000040E0324EA6EECCF03F0ED52EFCF6EF0DB
:101B700003C06FF06FC0EAFF6EC0E9FF6AC0E2FF0A
:101B800069C0E1FF6CC002F06BC001F0015202E0DD
:101B9000022A02D0025206E0E6CFEEFF012EFCD769
:101BA000022EFAD7186AF2BE188EF29E68C07CF038
:101BB0006CC07EF06BC07DF06DC07FF04EEC06F027
:101BC00018BEF28E015003D000D0000E016E41EF1E
:101BD0000FF0F86AD09E088EFE0E006E040E016EA5
:101BE000020EE96E000EEA6EEE6A002EFDD7012E9F
:101BF000FBD7600E006E040E016EA00EE96E040E9F
:101C0000EA6EEE6A002EFDD7012EFBD7EA6AE96A7A
:101C1000B8960C0EAF6EA60EAC6E900EAB6EC150A9
:101C2000C00B0F09C16E070EB46E196A1A6A236AD7
:101C3000040E246E0C0E256E266A2A6AC00EF2125D
:101C40002F0E926EA40E936E950E946EF9EF07F020
:101C500092988998686B68510EEC01F0682B00EC43
:101C600008F01D0E685DF7E17DEC08F0020E486E8D
:101C7000010E4926D8B04A2AD8B44B2AD8B44C2AE7
:101C8000000E81BA010E686F696F010E6A6F0F0E48
:101C90006C6F920E6B6F08D668C069F00F0E6B6F99
:101CA000800E6A6F21D601B07AD0010E686F6A6B20
:101CB000080E696F6C6B6B6B04EC08F002C04EF0A1
:101CC00001C04DF0686B68512AEC01F0682B00EC04
:101CD00008F00B0E685DF7E14EC068F0570E696FB3
:101CE0001BDE4DC068F0570E696F16DE010E686F7F
:101CF0006A6B420E696F6C6B6B6B04EC08F002C090
:101D000058F001C057F0686B68513FEC01F0682B48
:101D100000EC08F00B0E685DF7E158C068F0570E54
:101D2000696FFADD57C068F0570E696FF5DD4D52E7
:101D300002E14E520AE0686B6A6B050E696F300E65
:101D40006C6F6B6B04EC08F009D0686B6A6B050E66
:101D5000696F200E6C6F6B6B04EC08F04DC05CF08B
:101D6000686B4EC05BF057C05EF0686B58C05DF0AA
:101D70004D50535C09E14E50545C06E14D5202E176
:101D80004E5201E0632B02D0636B646B6351130806
:101D900002E2642B636B4EC054F04DC053F0E8EC8C
:101DA00007F0DED5DADD0152D8B46DD0010E686FD0
:101DB0001AD6015268E0010E686F6A6B340E696FC3
:101DC0006C6B020E6B6F8ED6686B685154EC01F031
:101DD000682B00EC08F0170E685DF7E134C068F07E
:101DE000370E696F99DD200E00EC08F0300E00EC24
:101DF00008F0780E00EC08F035C068F0370E696F17
:101E00008BDD0A0E00EC08F00D0E00EC08F03452E9
:101E100001E000D0355201E000D06151355C18E09E
:101E2000010EA96E35C0A8FFA69CA69EA684F2CF7F
:101E300000F0F29E0F01550EA76EAA0EA76EA682A5
:101E4000A6B2FED7A6940050F21200017DEC08F075
:101E50005BC02CF05CC02DF02E6A5DC02FF05EC020
:101E600030F0316A64C032F063C033F0010E686F45
:101E70006A6B2C0E696F6C6B080E6B6F020E6D6FC8
:0A1E800052D6015200E0F4D6030030
:020000040030CA
:0E00000000051E1F008381000FC00FE00F409F
:00000001FF
